:020000040000FA
:06000000000000003028A2
:080008006E2A28204320292064
:1000100063206220702020203220302030203320C6
:1000200050206320622020203320312030202020E7
:100030003120362046203820372033202020202031
:100040005820742061206C20320030002E003000D7
:1000500056206520722020203000300035002020FE
:10006000203084005F30FF008001840AFF0B3428B9
:10007000FF018B01831603138E309F0083128030A3
:100080009F001F14E1308316031385008312FF3095
:100090008316031386008312183083160313870018
:1000A0008312023083160313810083128312031319
:1000B00090018312031385018601870105152B2307
:1000C000E42602303527AE0004303527B100063073
:1000D0003527A90008303527D0000A303527CF0052
:1000E0000C303527EE000E303527EF001030352765
:1000F000F00012303527F10014303527D7000430D6
:10010000B3004124031830280130B400B22646263B
:100110000310600D0639A0006430BC000023870086
:100120003C08653C1E23633087003C0D1E23BC0B3E
:100130008E28B2264626B200BE00CE000230D8007D
:1001400002303E02031CA928281528140030B400F0
:10015000AB280130B4002414FF30F8007F228E0158
:1001600021309000831603138C1583120B178B1705
:100170000511640000308A0034088207C328EC2887
:10018000BD29CC29A82923110130B400281CD52869
:100190002810241502303E02031CDB2922163E08DB
:1001A000AF00BF013E08B200E928A81CDB29A81057
:1001B000241102303E020318DB29221EDB29221201
:1001C0003E08AF003208BF00281DE9282B23281164
:1001D000EA2836235923DB294626BE0063308700F0
:1001E0002319C328A31E01293F083E020319FB2837
:1001F00003185C294929A3122B23281D0129A814BF
:10020000C3281830230503190B29FF30BA00A3199E
:100210004929231A5C29FF30BA00241C1429061A24
:10022000192924102814C328061E19292414A814D7
:10023000C328861A22290301780703192829F80BF5
:1002400028292529FF30F8002829241D12291729DB
:10025000061D4929861D5C292310A3102210633036
:100260008700023060074E0203183D290301600732
:10027000031D60034E0203184629D80B44290515B7
:1002800064300D230511A2156008CE0041242B23F4
:10029000A729A310A31BA429231C7629BA0B522932
:1002A000FF30C0004008A7070319C001231F892998
:1002B0003E08AF005A2389292310231BA429A31C1D
:1002C0007C29BA0B6529FF30C0004008A707031935
:1002D000C001A31F89293E08AF005A23103027020E
:1002E0001030031C2708BA02BA03892923140130ED
:1002F000AC000230D8008129A314FF30AC000230DA
:10030000D8000130C0003E08AF002214A701E5016B
:10031000A1292C08AF07221C9F292F083E02031990
:100320009F29031895293E082F024C0203189F2984
:10033000291D9C29B30BA1290430B400A72904303E
:10034000B3000230B400A729A312A3112312DB29A2
:10035000633087002B23051518302305031DBC29A6
:10036000061DBC29861DBC2905112111A3122310CD
:10037000A3100130B400DB29DB29A21DC529A2117D
:100380000310600D57070639A000DA22211502304C
:10039000AD000330B400DB2926080F02031CDB2963
:1003A0008F00AD0BDA292B088700211105110130D0
:1003B000B400EC28DA221F19152A831603131E082D
:1003C0008312DB001E08DA007208DC007308DD000F
:1003D0005B08DD025A08031C013EDC02031CF629FF
:1003E0005A08F2005B08F30003300D2A7308F40288
:1003F000031CF3037208F302031CF20383160313B6
:100400001E088312F407031C082AF30A0319F20AD0
:100410001E08F3070318F20A0630F70277080319DB
:100420000130031C0130F7001F15C51C462A01309E
:10043000F700C51010304802031D242AA311003014
:100440004702031DA3153C2A11304802031D2E2A22
:10045000231200304702031D23163C2A12304802A3
:10046000031D3C2A00304702031D392A2814231596
:100470003C2AA81423153C2A141F3F2A14138C1D50
:10048000422A8C11831603138C158312211D6D2AA9
:10049000211F6A2AF70B6C2AA11C5B2A2B088700F4
:1004A000A110E50B582A051D572A0511582A0511D8
:1004B000250AF7006C2A2A088700051510100F0876
:1004C000A5001014A1142602F7000318682AF701EA
:1004D000F70A6C2A2B088700CC29B928E200030E02
:1004E0008301E1000A08E3008A01831203139122C9
:1004F00063088A00610E8300E20E620E0900363046
:1005000094008C11831603138030940060309100A6
:100510006830930083120313C601C5011308141336
:10052000080002308A0046088207992AA42AB32AC2
:10053000C02A8C1DCE2A8C111308831603131412A3
:10054000831203130130C6008C1DCE2A8C111308B0
:10055000C700CF22C900C90BB02A0330C600CE2A7B
:100560000230C600CE2A8C1DCE2A8C111308C8007A
:10057000C514831603138C1183120030C600CE2AD3
:1005800083160313141ECC2A831203138C1DC92A4D
:100590008C110030C600CE2A8312031308004708CE
:1005A0000739820702340234013401340134013442
:1005B00001340134A11DDE2A8023DF2A4123A60055
:1005C0000023AA002C08A0070023AB0010108E0106
:1005D0008F0110140800F600F022F60BEC2A080038
:1005E00064300D230515C8300D230511FA300D2395
:0805F000000000000800002BD0
:1006000003308A00073020058207A734A534E5347B
:10061000E434E634C634C7348734B800FA30B9005D
:100620006400122B132B142B152B162B172B182BA6
:10063000192BB90B102BB80B0E2B0800B800640057
:10064000212B222B232B242B252B262B272B282B2E
:10065000B80B1F2B08000430CC000512A111851522
:100660002117291C21132130900008000830CC00EC
:100670000516A11585112117A91C21130130900021
:10068000080003308A00F03027050F3003192708CF
:10069000820778347434743474346F346F346F3444
:1006A0006A346534603457344D3448343F3435341B
:1006B0003034A3163F083E02BA000318612BBA0972
:1006C000BA0A0310BA0C0230BA0708001E08D40098
:1006D000831603131E0883120313D5000800831624
:1006E00003131E0883120313D5071E080318013EC7
:0606F000D4070800802B76
:1007000003308A00F03027050F30031927088207CD
:100710008C346934553446343C3434342F342A34E0
:100720002534233420341F341E341C341C341B3431
:1007300078347434743474346F346F346F346A348E
:100740006534603457344D3448343F3435343034B4
:100750008C346934553446343C3434342F342A34A0
:100760002534233420341F341E341C341C341B34F1
:100770000330DA00A830DB000330DC008830DD0015
:100780005008B600CE2B0330DA009830DB0003307F
:10079000DC004930DD004F08B600CE2B1030BC0025
:1007A0003608B500B61FD62BB509B50A5A08D200CF
:1007B0005B08D300DB0A031DDE2BDA0A5527350858
:1007C000BB00B00103013B070319012C550EBC000F
:1007D000BC0C07303C05B007031CF02B05300D2482
:1007E000BB0BE62BB61BFB2B300AD507031CFA2BE1
:1007F000FF30D500012C300AD5020318012C05303A
:100800000D245C08D2005D08D300DD0A031D092C0D
:10081000DC0A7327BC0BD62B0800E100633087008D
:1008200061088B138B1B112CE1000130E300610880
:10083000E200051564300D230511FA300D23E20B9B
:10084000192CFA300D23FA300D23FA300D23FA302B
:100850000D23FA300D23631C0800172C002387009A
:1008600026080D2308002C08A0070023870003108A
:10087000260C0D232C08A0070023870026080D2333
:100880000800640004308A000608BC003C0D0639EC
:100890008207032E412CCF2D412C5B2C412C0000D4
:1008A000000003103D1C08003D10F02228118E228C
:1008B0008B17031408003D148B138B1B5C2CF02248
:1008C000061D702C861D722C061EAB2C861E832CDA
:1008D000061F9C2C06080339023C0319602C412C8E
:1008E0003623732C2B23B2264626BE00E0303E056D
:1008F00003197E2CBF0159238E2208003108BF0046
:1009000059238E2208002B23C8300D232530A60042
:10091000B2264626BE000030BE07031D952C0130CE
:10092000AC003324633087009B2CFF30AC003324B1
:10093000633087009B2C412C0430EB222215412C84
:1009400084001E088000831603131E0883120313FD
:10095000840A800008000A08CD00DC30B7000130AE
:10096000AC001330A6002B23B22670087202031DC0
:10097000BF2C3230A600710873020318C62C332432
:1009800063308700B70BB42C06300D24DC30B70081
:10099000FF30AC001330A6002B23B2267208DA0019
:1009A0007308DB006E08DC006F08DD009526031C71
:1009B000F12C7208DA007308DB006E08DC006F08A7
:1009C000DD001930DD070318DC0A95260318EA2C30
:1009D0003230A600332463308700B70BCD2C0330B0
:1009E0000D240130AC0036234B30A6000630A005A4
:1009F00020082E24633087002008023ED7009B3059
:100A0000B7009C26A210AE01D401D501732754086B
:100A1000D6005508D700A126CA01112D362333244C
:100A2000CA0108272B230A300D23B2266630A024E2
:100A300066230A300D23B2266830A0246F230A30C3
:100A40000D23B2266A30A0246F230A300D23B2266C
:100A50006C30A0246F23633087000310D40CD50CB6
:100A60000310D40CD50C6608DA006708DB006C08AC
:100A7000DC006D08DD009526DA1F432DDB09DA095D
:100A8000DB0A0318DA0A0330DB020301031C013E10
:100A9000DA02031C552D0C30CA07031C512D0430FB
:100AA0000D2432300D232E24132DA2185C2DA214F8
:100AB000023040272E082127AE0AA21C6F2D5408B1
:100AC000DA005508DB005608DC005708DD009526E3
:100AD00003186F2D22196E2D02300D24F022A21C56
:100AE000852D5408DA005508DB005608DC0057084D
:100AF000DD00DD0A031D7D2DDC0A95260318852DFA
:100B00002219842D09300D24F0225408DA005508EA
:100B1000DB005608DC005708DD005D08DB075C08D9
:100B20000318013EDA070130E4000310DA0CDB0C95
:100B3000E40B952D5A08D4005B08D5007327662373
:100B40005408D6005508D700A1265608DA005708E1
:100B5000DB007008DC007108DD0095260318B22D5B
:100B6000B70B0E2D2E08B100023035278312031368
:100B7000B10204304027310821270430D40000306E
:100B8000D500732702303527AE00143040275708B0
:100B900021274D088A008B17B2264626412C3D148A
:100BA0008B138B1BD02D0230EB22061DE72D861DEB
:100BB000EA2D861EF02D861EF32D061EED2D861EB7
:100BC000F62D06080339013C0319D52D412CD0031D
:100BD000B823F92DD00AB823F92DD001B823F92D67
:100BE000CF03C323F92DCF0AC323F92DCF01C3238C
:100BF000F92D08304027500821270A3040274F0898
:100C00002127F022412C3D148B138B1B042E033023
:100C1000EB22061D172E861D292E061E3B2E861E34
:100C20003D2E06080339003C0319092E412CB2263B
:100C30001E08EE00831603131E0883120313EF0031
:100C40000C3040276E0821270E3040276F082127DF
:100C50003F2EB2261E08F000831603131E088312CF
:100C60000313F1001030402770082127123040276D
:100C7000710821273F2E29153E2E29114126F022E9
:100C8000412C06304027290821270800C830DF0002
:100C900021120730D20097304107D3000318D20A3F
:100CA0004108E0005527F0305405031D672E7208F7
:100CB000DA007308DB005408DC005508DD005D082D
:100CC000DB025C08031C013EDA02031C702E211EAD
:100CD0006B2EA11E7D2EE00A4A27A1162116782E22
:100CE000211E742EA11A7C2EE0034F27A11221167B
:100CF000DF0B522E0830112CE0036008C1002313D3
:100D0000A3132E08E0020319872E03188B2E231736
:100D1000E0010301942E2E0831026002031C932E81
:100D2000A3173108E000600808005D08DB025C08DA
:100D3000031C013EDA0208000730D2009730D300CE
:100D40000800D30A53080319D20A08009E0C831620
:100D500003139E0C83129E0C831603139E0C1E0815
:100D6000831208001F151F19B32E1E08F2008316E8
:100D700003131E0883120313F30008003108B700A1
:100D80009C260030DA000030DB000030DC0005304B
:100D9000DD005A08D4005B08D50073275D08DB0727
:100DA0005C080318013EDA074A27B70BC92E043046
:100DB000DA000030DB005A3084000008D400840AD6
:100DC0000008D500732708008B138B1BE42E7F309F
:100DD00006020319F02E00303527AA3C031908003B
:100DE000F022F02200304027AA302127BE260B3007
:100DF000B7000330BC003C0840273527B0003C0357
:100E00004027300821270230BC07B70BFB2E080013
:100E10000A30F500FF30D100A00A002387005108F6
:100E20001E23A003A0030023870051081E23A00A4D
:100E30001430D102F50B0C2F0023870032300D2324
:100E40000800831203178C00831603178C130C15EC
:100E500055308D00AA308D008C140C1183160317A9
:100E60008C18302F831203130800831203178D0090
:100E7000831603178C130C1483120C080313080039
:100E8000831203178D0003130800831203178C00CD
:100E900003130800D30A031D0800D20A080001301A
:100EA000D30203180800D203080083120313530867
:100EB00003178D000313520803178F0083168C1736
:100EC0000C140000000083120C080313D500031754
:100ED0000E080313D400831603178C138312031315
:100EE00055080800D50083120313530803178D001B
:100EF0000313520803178F000313550803178C00C0
:100F00000313540803178E0083168C170C158312D5
:100F100003138B138316031755308D00AA308D00F1
:0E0F20008C14000000000C1183120313080053
:02400E00723FFF
:104200000000000004000400920092000500050078
:104210000000000000000000000000002600260052
:0C42200003000300E000E00000000000CC
:00000001FF
